:0A15AD000001020203030404050517
:10067200E4F513F512F511F510C212C20FC211C240
:100682001012081C7E117F008E438F44754B11752A
:100692004C1275411175421C754911754A3C754DD4
:1006A20011754E5CEE54E070030207B675140075C6
:1006B20015808E168F17C374869FFF74119ECF24E8
:1006C20002CF3400FEE48F0F8E0EF50DF50CF50B04
:1006D200F50AF509F508AF0FAE0EAD0DAC0CAB0B7C
:1006E200AA0AA909A808C3120C785026E515250BF9
:1006F200F582E514350AF58374CDF0E50B2401F596
:100702000BE4350AF50AE43509F509E43508F5087C
:1007120080C4E4F50BF50AF509F508AF0FAE0EAD8E
:100722000DAC0CAB0BAA0AA909A808C3120C78508D
:1007320031AE0AAF0BE5172FF582E5163EF583E0E1
:10074200FDE5152FF582E5143EF583EDF0EF24016A
:10075200F50BE43EF50AE43509F509E43508F50838
:1007620080B985144385154474002480FF741134C4
:10077200FFFEC3E54C9FF54CE54B9EF54BC3E546AA
:100782009FF546E5459EF545C3E5489FF548E54793
:100792009EF547C3E5429FF542E5419EF541C3E51B
:1007A2004A9FF54AE5499EF549C3E54E9FF54EE558
:1007B2004D9EF54DD2E843D82090E668E04409F01A
:1007C20090E65CE0443DF0D2AF90E680E020E105A7
:1007D200D21312134190E680E054F7F0538EF8C220
:1007E2001230100512044EC2103012291216815016
:1007F20024C212121494200F1690E682E030E7040D
:10080200E020E1EF90E682E030E604E020E0E4124E
:0A08120010D412168312167E80C760
:10044E0090E6B9E070030204FF14700302057C24E9
:10045E00FE70030205FF24FB70030204F9147003FF
:10046E000204F31460731460762405600302065EC2
:10047E00121685400302066A90E6BBE024FE602257
:10048E0014603324FD601114602224067048E54385
:10049E0090E6B3F0E5448037E54B90E6B3F0E54CDB
:1004AE00802DE54590E6B3F0E5468023E54790E6DE
:1004BE00B3F0E548801990E6BAE0FF121370AA0671
:1004CE00A9077B01EA494B600DEE90E6B3F0EF9081
:1004DE00E6B4F002066A02066312156902066A1293
:1004EE00161E02066A12125902066A1215570206E3
:1004FE006A121687400302066A90E6B8E0247F600F
:10050E001514601924027063A20FE43325E0FFA2D4
:10051E0011E4334F8041E490E740F0803F90E6BC19
:10052E00E0547EFF7E00E0D394807C0040047D0189
:10053E0080027D00EC4EFEED4F24ADF58274153E2B
:10054E00F583E493FF3395E0FEEF24A1FFEE34E64E
:10055E008F82F583E0540190E740F0E4A3F090E63B
:10056E008AF090E68B7402F002066A020663121697
:10057E0089400302066A90E6B8E024FE6016240263
:10058E00600302066A90E6BAE0B40105C20F0206E5
:10059E006A02066390E6BAE0705590E6BCE0547EBF
:1005AE00FF7E00E0D394807C0040047D0180027DBC
:1005BE0000EC4EFEED4F24ADF58274153EF583E44E
:1005CE0093FF3395E0FEEF24A1FFEE34E68F82F524
:1005DE0083E054FEF090E6BCE05480131313541FD6
:1005EE00FFE0540F2F90E683F0E04420F0806D8002
:1005FE006412168B506690E6B8E024FE6019240251
:10060E00705A90E6BAE0B40104D20F804F90E6BA69
:10061E00E064026047803E90E6BCE0547EFF7E00C0
:10062E00E0D394807C0040047D0180027D00EC4E7E
:10063E00FEED4F24ADF58274153EF583E493FF3342
:10064E0095E0FEEF24A1FFEE34E68F82F58380085D
:10065E00120080500790E6A0E04401F090E6A0E082
:03066E004480F0D5
:010671002266
:03003300020CFCC0
:040CFC0053D8EF32A8
:101100001201000200000040C0161E08000001028B
:1011100000010A0600020000004001000902200050
:1011200001010080320904000002FF0000000705F1
:1011300001024000000705820200020009022000AF
:1011400001010080320904000002FF0000000705D1
:101150000102400000070582024000000403090468
:101160001003510048005900430041004D00530056
:1011700016035100480059002D00310020002000C6
:081180005600310032000000AE
:10090D0060801800010301010101010700000002D0
:10091D00000002001332120A080C0800000000004B
:10092D000000003F02030202020202070000000263
:10093D000000020013320A12100C08000000000023
:10094D000000003F033A0A0A0A0A030700000002EA
:10095D00000002001332120A080C0800000000000B
:10096D000000003F033A0A0A0A0A030700000002CA
:10097D000000020013320A12100C080000000000E3
:10098D000000003F602418870000000000000000F8
:10099D00000000000000000000000000000000004A
:1009AD0000000000000000000000000047188080DB
:0609BD00000000CA4E001C
:100ABB0090E60174CAF090E6F574FFF0901880E0B0
:100ACB0090E6F3F0901881E090E6C3F0901882E086
:100ADB0090E6C1F0901883E090E6C2F0901885E0A4
:100AEB0090E6C0F0901886E090E6F4F075AF0774CE
:100AFB0018F59A7400F59B759DE4E4F59EFF90E65E
:100B0B007BE090E67CF00FBF80F490E67174FFF011
:100B1B00F5B490E672E04480F043B680000000E448
:100B2B0090E6C4F000000090E6C5F0901887E090C6
:100B3B00E6C6F0901888E090E6C7F0901889E09030
:100B4B00E6C8F090188AE090E6C9F090188BE09018
:100B5B00E6CAF090188CE090E6CBF090188DE09000
:0B0B6B00E6CCF090188EE090E6CDF094
:010B7600225C
:03004300020D00AB
:03005300020D009B
:100D00000214D20002151800021502000214EA00B3
:100D100002130B000212960002168D0002168E00BE
:100D200002168F00021690000216910002146E0047
:100D30000216920002169300021694000216950005
:100D40000216960002168E000216970002169800F0
:100D50000216990002169A0002169B0002169C00C9
:100D600002169D0002168E0002168E0002168E00DC
:100D700002169E0002169F000216A0000216A10095
:100D80000216A2000216A3000216A4000216A50075
:100D90000216A6000216A7000216A8000216A90055
:100DA0000216AA000216AB000216AC000216AD0035
:080DB0000216AE000216AF00AE
:1010D40090E682E030E004E020E60B90E682E03027
:1010E400E119E030E71590E680E04401F07F147EDA
:0C10F400001211D290E680E054FEF022C1
:1014940090E682E044C0F090E681F04387010000CA
:0414A4000000002222
:1013410030130990E680E0440AF0800790E680E0DF
:101351004408F07FDC7E051211D290E65D74FFF047
:0F13610090E65FF05391EF90E680E054F7F022B2
:02137000A907CB
:10137200AE4DAF4E8F828E83A3E064037017AD0132
:1013820019ED7001228F828E83E07C002FFDEC3EEE
:09139200FEAF0580DF7E007F0044
:01139B00222F
:1011D2008E1C8F1D90E600E054187012E51D24014C
:1011E200FFE4351CC313F51CEF13F51D801590E6C3
:1011F20000E05418FFBF100BE51D25E0F51DE51CAE
:1012020033F51CE51D151DAE1C7002151C4E600544
:061212001214A880EE2278
:1014A8007400F58690FDA57C05A3E582458370F957
:0114B8002211
:1009C300C106C1880224000002390000023700007A
:1009D300022B1040022E0000C107C103023D025743
:0409E300023B0000D3
:10081C0090E600E054E74410F00000000000009067
:10082C00E61074A0F000000090E60B7401F090E666
:10083C001274E0F0000000E490E613F00000009069
:10084C00E614F000000090E615F000000090E618A9
:10085C00740CF000000090E6D27402F090E6047480
:10086C0080F00000007402F0000000E4F0000000D2
:10087C00120ABBE490E671F075B4FF90E672F07565
:10088C00B6FF75B1FF90E670F075B2FFD286F5B584
:10089C0012158B752402752500C3E4952CFF74107A
:1008AC00952BAD0790E630F0AF05EF90E631F0E414
:1008BC00F539F53AF537F53890E65EE04408F00086
:1008CC000000E490E68DF07FAAFE1215DF12139C57
:1008DC00C284C283D282C2807FAA7E001215DF53EB
:1008EC00B1EF7527007528B4753301753490752BED
:1008FC0010752CB875350675362CE4F52D53B17F73
:01090C0022C8
:03167E00020E5FFA
:02168100D32272
:02168300D32270
:02168500D3226E
:1012590090E680E030E71800000090E6207402F084
:10126900000000E490E621F0000000D2088016009A
:101279000000E490E620F000000090E6217440F0C0
:0D128900000000C20890E6BAE0F532D32262
:1015570090E740E532F0E490E68AF090E68B04F0FD
:02156700D3228D
:08161E0090E6BAE0F526D322A4
:1015690090E740E526F0E490E68AF090E68B04F0F7
:02157900D3227B
:02168700D3226C
:02168900D3226A
:02168B00D32268
:10008000E4F518F51990E6B9E0244D607814700392
:1000900002014D1470030201A914700302035E14DF
:1000A000700302039524F670030203B11470030277
:1000B00003FC2410600302044AE4F537F53890E6A7
:1000C0000B04F000000090E6047480F0000000745F
:1000D00002F000000090E60174C8F000000090E615
:1000E000C3743FF000000090E6C274FFF00000000F
:1000F000F5B5E4F5B0F5B37F82FE1215DF90E74069
:1001000074B202019CE490E68AF090E68BF090E6EF
:10011000A0E020E1F990E68BE0F518E4F539F53A36
:10012000F5B5F5B390E60174CAF0E490E6C3F0903B
:10013000E6C2F0D206D20400000090E6047480F01B
:100140000000007402F0000000E40203A6E4F53DA4
:10015000F53EF53BF53C90E60B04F000000090E620
:10016000047480F00000007402F000000090E601CA
:1001700074C8F000000090E6C3743FF000000090E7
:10018000E6C274FFF0000000F5B5E4F5B0F5B37F0A
:10019000AAFE1215DFD20690E74074B4F0E490E6B0
:1001A0008AF090E68B040203A6E490E68AF090E6DB
:1001B0008BF090E6A0E020E1F990E68BE0F518D313
:1001C00094174024E4F51974402519F582E434E7C6
:1001D000F583E0FF74AB2519F582E43418F583EF5D
:1001E000F00519E519B418DF90E6A0E04480F07F2F
:1001F0008C7E001215DF9018ABE0FF7E001215E830
:100200009018ABE0FF7E001215F19018ABE0FF7E76
:10021000001215FA9018B2E075F004A4FFAEF012C7
:1002200016039018B2E075F004A4FFAEF012160C9D
:100230009018B2E075F004A4FFAEF01216159018F5
:10024000B0E0FF5480C4131313540124FF9205EF50
:100250005440C41313540324FF920BE05402C313FD
:1002600024FF920C9018AFE0FF5480C41313135472
:100270000124FF920AEF5440C41313540324FF9245
:100280000EE0FF5408131313541F24FF9200EF5481
:10029000041313543F24FF9201E05402C31324FFBC
:1002A000920DA205928520001090E6C0200A0574E8
:1002B0004EF08013749CF0800E90E6C0200A057406
:1002C0009FF08003749DF09018B1E0FF7004C209A4
:1002D000C202EFB40104C209D202EFB40204D2098F
:1002E000C2029018B5E0FEA3E07C002400F528ECE3
:1002F0003EF527A3E0FEA3E02400F534EC3EF53301
:10030000A3E0FEA3E02400F52CEC3EF52BA3E0FED9
:10031000A3E02400F536EC3EF535A3E0FEA3E0248F
:1003200000F531EC3EF530A3E0F52DA3E0FEA3E0AF
:100330002400F52AEC3EF529E52D7006753F03757E
:10034000400CE52DB40106753F01754086E52D642E
:1003500002600302044CF53F7540C302044CE4F50F
:100360001974AB2519F582E43418F583E0FF744065
:100370002519F582E434E7F583EFF00519E519B4A2
:1003800018DF000000E490E68AF000000090E68BA1
:10039000741802043DC20690E74074B7F0E490E69A
:1003A0008AF090E68B04F090E6A0E04480F002042E
:1003B0004CE490E68AF090E68BF090E6A0E020E135
:1003C000F990E68BE0F518D394024024E4F5197413
:1003D000402519F582E434E7F583E0FF74C325195D
:1003E000F582E43418F583EFF00519E519B403DF5D
:1003F00090E6A0E04480F012139C805090E7407497
:1004000056F0A37403F0A3F0A3741BF0A37402F0DE
:10041000A37454F0A37402F0A314F0A37459F03041
:100420000805E4A3F0800690E74974FFF00000009F
:10043000E490E68AF000000090E68B740AF090E603
:0D044000A0E04480F01213C78002D322C355
:01044D00228C
:1014D200C0E0C083C082D2105391EF90E65D7401E8
:0814E200F0D082D083D0E0328B
:10150200C0E0C083C0825391EF90E65D7404F0D0D6
:0615120082D083D0E0321C
:10151800C0E0C083C0825391EF90E65D7402F0D0C2
:0615280082D083D0E03206
:10130B00C0E0C083C082854945854A4685468285B3
:10131B004583A37402F08541478542488548828501
:10132B004783A37407F05391EF90E65D7410F0D0F0
:06133B0082D083D0E032F5
:1014EA00C0E0C083C082D2125391EF90E65D7408C7
:0814FA00F0D082D083D0E03273
:10129600C0E0C083C08290E680E030E7208541450B
:1012A600854246854682854583A37402F085494773
:1012B600854A48854882854783A37407F05391EF92
:0D12C60090E65D7420F0D082D083D0E0323D
:01168D00322A
:01168E003229
:01168F003228
:011690003227
:011691003226
:10146E00C0E0C083C082C2AF75230000000090E6CA
:10147E008DE4F05391EF90E65FE04408F0D2AFD0E8
:06148E0082D083D0E032A1
:011692003225
:011693003224
:011694003223
:011695003222
:011696003221
:011697003220
:01169800321F
:01169900321E
:01169A00321D
:01169B00321C
:01169C00321B
:01169D00321A
:01169E003219
:01169F003218
:0116A0003217
:0116A1003216
:0116A2003215
:0116A3003214
:0116A4003213
:0116A5003212
:0116A6003211
:0116A7003210
:0116A800320F
:0116A900320E
:0116AA00320D
:0116AB00320C
:0116AC00320B
:0116AD00320A
:0116AE003209
:0116AF003208
:0609E8008F1A8C1B8D1C10
:1009EE0075B6FF75B5FF53B07F531A0753B1FE7F2F
:1009FE00647E001210C8E4F51DF51EC37402951E28
:100A0E00FFE51AA807088002C313D8FC30E005439F
:100A1E00B102800353B1FD7F647E001210C843B152
:100A2E00047F647E001210C853B1FB7F647E0012F7
:100A3E0010C8051EE51E7002051DC39403E51D6456
:100A4E0080948040B6E4F51DF51EC37409951EFF13
:100A5E00E51CAE1BA807088005CEC313CE13D8F92C
:100A6E0030E00543B102800353B1FD7F647E001276
:100A7E0010C843B1047F647E001210C853B1FB7FCF
:100A8E00647E001210C8051EE51E7002051DC3947B
:100A9E000AE51D6480948040B143B1017F647E00FD
:0D0AAE001210C853B1FE7F647E000210C814
:0915DF00AD07AC06E4FF0209E8C7
:0915E800AD07AC067F040209E81E
:0915F100AD07AC067F050209E814
:0915FA00AD07AC067F060209E80A
:09160300AD07AC067F010209E805
:09160C00AD07AC067F020209E8FB
:09161500AD07AC067F030209E8F1
:1010850012158B7F0A7E001210C81215CB7F027EC7
:10109500001210C812154D7F027E001210C81216DC
:1010A5007A7F027E001210C81215A97F027E0012F7
:1010B50010C81215817F027E001210C81215D57F47
:0310C500027E00A8
:0C10C800EF4E6007EF1F70F81E80F5224D
:0716260053A0F753A0DF22DF
:07162D0053A0F743A02022A7
:0716340043A00843A020229F
:07163B0053A0FE53A0FB22A7
:0716420053A0FE43A00422A7
:0716490043A00143A00422AD
:071597007F037E001210C863
:04159E0053A07F22B5
:0715A2007F037E001210C858
:0415A90043A08022B9
:04167A0053A0BF2298
:1014B9001215CB12154D12167A1215A91215811291
:0514C90015D512159E6F
:0414CE0043A04022D5
:0716500053A0F753A0EF22A5
:0716570053A0F743A010228D
:07165E0043A00843A0102285
:0716650053A0FE53A0FD227B
:07166C0053A0FE43A002227F
:0716730043A00143A0022285
:0A15B70053A0F753A0DF53A0EF226A
:0A15C10053A0FE53A0FB53A0FD222F
:06157B0012167A1215A9F8
:0A15810053A0F743A02043A010225E
:0A15CB0053A0FE43A00443A0022237
:0A1543001215CB7F037E001210C8C2
:0A154D0043A00843A02043A0102291
:0A15D50043A00143A00443A002223A
:0C158B0012158112159E1215D50214CE07
:1012D30012108512159E7F147E001210C81215B7C6
:1012E3001210C41214CE7F047E001210C81215818E
:1012F3001215437F1412109E12159E1210C412145D
:08130300CE7F0A7E000210C833
:1011880012108512159E1210C41214CE1210C41219
:1011980015CB1210C412154D1210C412167A7F14F2
:1011A8007E001210C81215C11215A27F037E00120C
:1011B80010C81215CB7F141210B212159E1210C44B
:0A11C8001214CE7F147E000210C83E
:1013F20012158B1210C4E4FFFE12154D1215CB12FA
:1014020015A912167A1214C512154D1215CB0FBF5B
:0914120000010EBE04E3BF0EE070
:01141B0022AE
:030CDE00120CE114
:100CE1007F0A7E001210C87F0212108A12159E120E
:0B0CF10010C41214CE1210C4D28022D6
:100B770012158B7F057E001210C8E4FFFE1214B910
:100B87000FBF00010EEF64034E70F27F0A7E001262
:100B970010C81215437F037E001210C812167A7F01
:100BA700037E001210C812163B1215A27F037E00A7
:100BB7001210C81216427F037E001210C81215D5F4
:100BC7001215811215977F037E001210C812162680
:100BD7007F037E001210C81214CE7F037E0012100E
:100BE700C812162D1215461215CB1215A212167A17
:100BF7007F037E001210C81215811215D5121597A2
:100C07001214CE7F037E001210C87F0A7E001210D6
:100C1700C8E4FEFF1214B90FBF00010EEF64034EC4
:090C270070F27F057E000210C886
:1014460012158B1215CB12154D12157BD28712145D
:10145600C81214B91215CB12154DC28712157B127C
:0814660015D512159E0214CEEB
:1012180090E60174C8F090E6C3743FF090E6C2749B
:10122800FFF0F5B4EF4E601675B00475B00675B0F2
:101238000675B00A75B00AEF1F70E91E80E675B42E
:10124800BF90E60174CAF0E490E6C3F090E6C2F0FD
:011258002273
:10152E00E4FFFED287D287C2870FBF00010EBE0135
:04153E00F2BF04EF05
:011542002286
:10139C00E4F51AF51BD2847F0A7E001211D2C284A6
:1013AC007F0A7E001211D2051BE51B7002051AC3C1
:0A13BC009405E51A6480948040DB7C
:0113C6002204
:1013C700E4F51AF51BD2837F0A7E001211D2C2837D
:1013D7007F0A7E001211D2051BE51B7002051AC396
:0A13E7009405E51A6480948040DB51
:0113F10022D9
:0116B0002217
:0116B1002216
:100DB80053B17FC284C283C2821215A912154D2075
:100DC8000D0312152E300B02C2861216B0200C6CC1
:100DD8009018ACE075F040A485F01AF51BAF237E9F
:100DE80000AC1AAD1B120C30D3EF9400EE94004007
:100DF800117F007E041211D2E51B151B70DF151A36
:100E080080DB9018ADE0751A00F51BAF237E00ACAF
:100E18001AAD1B120C30D3EF9400EE940040117FF2
:100E2800007E011211D2E51B151B70DF151A80DB3D
:100E38009018AEE0FF7E001211D28009752301E5FB
:100E480023640160FA1216B1300B09D2867F647EE2
:060E5800001211D2D28449
:010E5E002271
:040EFF008E188F19A1
:100F0300E51945187039752301120DB8200D031228
:100F130013F2200E0A2001028008121188800612A3
:100F230011881212D3E4FDFCC3ED9528EC952750EC
:100F33000A120CE10DBD00010C80EDD284C283E5E1
:100F43001964014518700343B180E51965407004C5
:100F5300E518653F702430020C1215A912154D12C5
:100F63000DB81213F2200E08200108121188800612
:100F73001211881212D3D284C283E5402401FFE404
:0E0F8300353FFEEFB51907EEB5180343B180F8
:010F9100223D
:10141C00AB070000007F007C017D00120C4290E6BF
:10142C00D0EFF0000000EB90E6D1F000000075BBAF
:0A143C0004000000E5BB30E7FB22CE
:100E5F00200603020EFEE5BB20E703020EFE200470
:100E6F0003020EFEAF3AAE39120EFF000000E52B63
:100E7F0090E6D0F0000000E52C90E6D1F0000000E5
:100E8F00C284C28375BB04000000E5BB20E706D215
:100E9F0084C28380F5C284C283E52D7003120CE1F6
:100EAF00E52DB40103120CDEE52DB40209120CDEA0
:100EBF00120CE1120CE1053AE53A70020539C395BF
:100ECF0036E53995354028C204AF31AE3012141CC7
:100EDF00E4FDFCC3ED9534EC9533500A120CE10D93
:0F0EEF00BD00010C80ED53B17FC284C283D2825B
:010EFE0022D1
:10101E00300663E5BB30E75E30045BE53A45397078
:10102E0009120DB81213F2120B77000000E52B9087
:10103E00E6D0F0000000E52C90E6D1F0000000C2F2
:10104E0084C28375BB04000000E5BB20E706D28492
:10105E00D28380F5C284C283121446053AE53A70F3
:10106E00020539C39536E5399535400A53B17FE40B
:07107E00F539F53AC2042226
:0116B2002215
:0116B3002214
:03000000020F925A
:0C0F9200787FE4F6D8FD75814E020FD97F
:100C3000EF8DF0A4A8F0CF8CF0A428CE8DF0A42ED8
:020C4000FE2292
:100C4200C2D5EC30E709B2D5E4C39DFDE49CFCEECD
:100C520030E715B2D5E4C39FFFE49EFE120C89C3B0
:100C6200E49DFDE49CFC8003120C8930D507C3E4AB
:060C72009FFFE49EFE223C
:100C7800EB9FF5F0EA9E42F0E99D42F0E89C45F0D2
:010C88002249
:100F9E00020672E493A3F8E493A34003F68001F2F1
:100FAE0008DFF48029E493A3F85407240CC8C33354
:100FBE00C4540F4420C8834004F456800146F6DF23
:100FCE00E4800B010204081020408090090DE47E9D
:100FDE00019360BCA3FF543F30E509541FFEE49318
:100FEE00A360010ECF54C025E060A840B8E493A3DF
:100FFE00FAE493A3F8E493A3C8C582C8CAC583CA0A
:10100E00F0A3C8C582C8CAC583CADFE9DEE780BEC1
:0109E700000F
:100C8900BC000BBE0029EF8DF084FFADF022E4CC4F
:100C9900F875F008EF2FFFEE33FEEC33FCEE9DEC18
:100CA900984005FCEE9DFE0FD5F0E9E4CEFD22ED5E
:100CB900F8F5F0EE8420D21CFEADF075F008EF2FA8
:100CC900FFED33FD4007985006D5F0F222C398FD99
:050CD9000FD5F0EA2236
:00000001FF
